:104EEB001256A253B1F8126319306720C2671266CB
:104EFB00061267941264EC1260C91259CA125E4B07
:104F0B00126349124F631244281265F2306622C2B3
:104F1B0066121FE912537812657F126529126546D6
:104F2B001251F540031246C91265DD123B50124A6D
:104F3B00DE12646012672512583F123C2312564C46
:104F4B00126053900206E524F0A3E525F0A3E522B9
:084F5B00F0A3E523F0808C2295
:105F16009003867401F07E027F3C7B40E4FD1263B1
:105F2600767E027F0A7B14E4126376900224740A5A
:105F3600F0A374ABF0A3740AF0A374ABF0C22CC246
:105F46002D9003A07402F0D22ED27590027C74506C
:025F5600F02237
:1046C9007FFE7E011263A0501F7B007A02E4FDFC8D
:1046D900FFFE1253197FFE7E031263A0402CE4FDF6
:1046E900FF7E0212489D80227FFE7E031263A05046
:1046F900167B007A02E4FDFCFF7E02125319E4FDE9
:10470900FFFE12489D8003D26822900000E0F52048
:10471900A3E0F521900238E520F0A3E521F090000F
:10472900B61215FD90022C1216159000CAE0FFA3CF
:10473900E0900236CFF0A3EFF0E52154072403F50A
:104749001364056005E513B40A04E4F51422E513BE
:1047590064046005E513B409047514012275140293
:01476900222D
:10650B00C2AFD2ACC086758640C28FD086D2AD43A7
:0E651B00BA6043E840E4F5D843A908D2AF22A5
:10102E007580F875E18F75E9C875908075E27F75EA
:10103E00EA8075A0E075E33F75EBC075B01975E4F5
:05104E00E675EC19221B
:1056A200E4FF12579D12102E1262B31246C9125F06
:1056B200167D057C007F441236F17F807E251249DB
:1056C200347F641261047D647FA07E0F124D7412D8
:1056D2004BEC12675C4002D24C1260173007121278
:1056E2004DF54002D23A7E037F781249C54002D27C
:0556F2007212650B229D
:10648500EFB4200E205503305819E4FF12579DD262
:106495005722EFB4400D205503305807E4FF12573B
:0464A5009DD257220B
:1064A900D265900399E004F0C3940A4004E4F0D261
:1064B90067900398E004F0C394C84004E4F0D266FE
:0464C900124627222E
:105F9900D3EF9450EE940040037F0522D3EF943C55
:105FA900EE940040037F0422D3EF9428EE9400403E
:105FB900037F0322D3EF9414EE940040037F02225F
:0F5FC900D3EF9400EE940040037F01227F00226B
:10662E00306B0F90038EE004F0C394644004E4F0EA
:03663E00C26B220A
:10442800302A1490038CE004F0C3940A400BE4F0A3
:10443800A2B5B392B58002C2B5306C1490038DE07A
:1044480004F0C39405400BE4F0A2A0B392A080024C
:10445800C2A0306B67900234E0FEA3E0FF125F99C0
:10446800EF700D206C02C2A0C2A1C2A2C2A3C2A456
:10447800EFB40107206C52D2A0804EEFB40209209D
:104488006C02D2A0D2A18041EFB4030B206C02D2FF
:10449800A0D2A1D2A28032EFB4040D206C02D2A027
:1044A800D2A1D2A2D2A38021EF6405701C206C0295
:1044B800D2A0D2A1D2A2D2A3D2A4800D206C02C2D3
:0C44C800A0C2A1C2A2C2A3C2A412662E10
:0144D40022C5
:1053D500C22CC22DC22E9003A0E0701804F0D22D6D
:1053E50090008AE0FEA3E0FF90008DE0FD124D7471
:1053F50043B701229003A0E0B401167402F0D22E47
:1054050090008AE0FEA3E0FF7D64124D7443B7016E
:1054150022E49003A0F0D22C90008AE0FEA3E0FFE6
:0C54250090008CE0FD124D7443B7012292
:1063190030742CC274E50824FE600F24F160161451
:106329006010241170191253D522D26BE490038E98
:10633900F022D25522B26C306C03C28322D283225E
:10613D00305734C257305824E4FF12579DD2AFC2A6
:10614D0058E490038FF07F01125C1AD2ACD2ADD21D
:10615D00CE7F701265B11266FF12668DE490038FCB
:08616D00F0A3F0900380F02282
:1064CD0053B1F8C2AF206C02C2A0C2A1C2A2C2A336
:0F64DD00C2A4D283E4FF1265C81263EE80E222EC
:105ED300206C02C2A0C2A1C2A2C2A3C2A4D283C226
:105EE3006C1266A01267127F7012674AC2CE53B754
:105EF3007E302904D2A58002C2A57F01125C1AC29A
:105F0300AFC2ACC2ADE4F5D87F8012579DD2AF12B9
:035F13006788227A
:104ADE00305608305B05C256D2552230161490005F
:104AEE002AE0FF900390E004F0C39F406AEFF0D2FB
:104AFE005522206B5B202A50202B4D30191490002C
:104B0E002AE0FF900390E004F0C39F404AEFF0D2FA
:104B1E005522E4900390F0A21272107218721A725B
:104B2E001172137219721B721C7215726C401390F3
:104B3E00002AE0FF90038FE004F09F401AEFF0D2BE
:104B4E005822E490038FF022E490038FF0A3F0221A
:084B5E00E490038FF0A3F022A4
:10605300205826205523C2AFA273727472697257F7
:10606300725C72677266400D900391E06412600582
:10607300D2AF12677CD2AF800E3055051264CD804B
:0B60830006305803125ED312613D226C
:105B8A0000000030006200750000008A008F009A51
:105B9A0000A300AB00CD00D100FE00000000000011
:105BAA00000000000020005000820095000000AABA
:105BBA0000AF00BA00C300CB00ED00F1011E0000E7
:085BCA000000000000000000D3
:10673800900A02E07006C29C75995A22C29C75990B
:02674800FF222E
:084B66009002B7EEF0A3EFF09E
:104B6E007B017A0A7900900A02E02403FD12656344
:104B7E00900A02E02403F582E4340AF583E06F70B4
:104B8E0057FF900A02E0FEEFC39E502953B1F8740E
:104B9E00032FF582E4340AF583E0FE9002B7E0FCC1
:104BAE00A3E0F5828C83EEF09002B7E475F001126B
:104BBE0014330F80CDE4900068F0A3F0A3F0A3F0BF
:104BCE00A3F0A3F090007BF0A3F0A3F0D26A9003C1
:0D4BDE009EF0C29C75995A22C29C7599FFE9
:014BEB0022A7
:104E7200900A02E0D3948C4002E4F0E4900068F0DF
:104E8200A3F0A3F0A3F0A3F0A3F090007BF0A3F0B3
:104E9200A3F0FD900A02E0FCEDC39C501D53B1F853
:104EA2008F828E83E0FB74032DF582E4340AF5834E
:104EB200EBF00FBF00010E0D80D97B017A0A790059
:104EC200EC2403FD126563900A02E02403F582E4F8
:104ED200340AF583EFF0C29C900383E02400F5824C
:084EE200E4340AF583E0F599C0
:014EEA0022A5
:105D38007B017A0A7900900A02E02403FD12656368
:105D4800900A02E02403F582E4340AF583E0B507FB
:105D58001E900A04E0FFB441089003917412F08089
:105D680006EFB40502D256C25BC29C75995A22C28C
:055D78009C7599FF225B
:106175007B017A0A7900900A02E02403FD12656327
:10618500900A02E02403F582E4340AF583E0B507BA
:1061950010900A03E0900381F0C25BC29C75995A86
:0761A50022C29C7599FF2244
:1031DC00900A01E0FF12165E3230013230023230BA
:1031EC0003323004323005323006323007323008C8
:1031FC0032300932300A32410B32510C32590D3215
:10320C00610E32690F3249103271113279123281EA
:10321C001332891432911532991632A11732A9182A
:10322C00000032B1EF25E02408F582E43402AF82CD
:10323C00FE124E72227E027F1E124E72227E027F80
:10324C0020124E72227E027F24124E72227E027F48
:10325C0026124E72227E027F28124E72227E027F2E
:10326C002A124E72227E027F2C124E72227E027F16
:10327C0030124E72227E027F34124E72227E027FF8
:10328C0036124E72227E027F06124E72227E027F10
:10329C0008124E72227E027F38124E72227E027FFC
:1032AC003A124E7222900A02E0C394804005D23B3F
:1032BC00D23D22900A01E0B4780C900381E0B40C6A
:1032CC0005D23BD23822900A01E0B47822900381D7
:1032DC00E025E0248AF582E4345BF583E493FE7404
:1032EC000193FF9002B5EEF0A3EFF0124E72229014
:1032FC000A01E0B47921900381E025E024AEF58247
:10330C00E4345BF583E493FE740193FF9002B5EE15
:07331C00F0A3EFF0124E7266
:013323002287
:10574B007B017A0A7900900A02E02403FD1265635B
:10575B00900A02E02403F582E4340AF583E06F70CB
:10576B002B900A03E0FEA3E0FDEEEDFF900350EE5D
:10577B00F0A3EFF04E7006C29C7599FF22D2739086
:10578B00034BE04401F0C29C75995A22C29C759957
:02579B00FF22EB
:103CE4007B017A0A7900900A02E02403FD126563DD
:103CF400900A02E02403F582E4340AF583E06F605D
:103D040003023D9B900A04E0FFE4FCFDFE781012E0
:103D140015EAC004C005C006C007900A03E0FFE42A
:103D2400FCFDFE78181215EAD003D002D001D000B1
:103D3400121581C004C005C006C007900A05E0FF43
:103D4400E4FCFDFE78081215EAD003D002D001D0BD
:103D540000121581A804A905AA06AB07A3E0FFE495
:103D6400FCFDFE1215819003471216159002A1E086
:103D74007002A3E0600C9003471215FDEC4D4E4F0A
:103D84007006C29C7599FF22D27390034BE04410D5
:0D3D9400F0C29C75995A22C29C7599FF22BD
:1061AC007B017A0A7900900A02E02403FD126563F0
:1061BC00900A02E02403F582E4340AF583E0B50783
:1061CC000FD27390034BE04420F0C29C75995A2275
:0661DC00C29C7599FF2230
:105AF8007B017A0A7900900A02E02403FD126563AB
:105B0800900A02E02403F582E4340AF583E06F701A
:105B180022D273900A03E0FEA3E0FDEEEDFF9003AE
:105B28004CEEF0A3EFF090034BE04404F0C29C75F8
:095B3800995A22C29C7599FF22C2
:105B41007B017A0A7900900A02E02403FD12656361
:105B5100900A02E02403F582E4340AF583E06F70D1
:105B610022D273900A03E0FEA3E0FDEEEDFF900365
:105B71004EEEF0A3EFF090034BE04408F0C29C75A9
:095B8100995A22C29C7599FF2279
:1056F7007B017A0A7900900A02E02403FD126563B0
:10570700900A02E02403F582E4340AF583E06F701F
:105717002DFF74032FF582E4340AF583E0FE7452FB
:105727002FF582E43403F583EEF00FEFB407E3D2ED
:105737007390034BE04480F0C29C75995A22C29C37
:035747007599FF52
:01574A00223C
:10458000900A01E012165E45AC1845B07745CC782C
:1045900045EE7945B8A045C0A145C4A245B4A345A0
:1045A000BCA445C8AF4610B000004626125D3822B4
:1045B00012617522123CE42212574B221261AC2286
:1045C000125AF822125B41221256F722900381E020
:1045D00025E0248AF582E4345BF583E493FE7401DC
:1045E00093FF9002B5EEF0A3EFF0124B662290031A
:1045F00081E025E024AEF582E4345BF583E493FEAC
:10460000740193FF9002B5EEF0A3EFF0124B662217
:10461000900A03E0B4550AD23BD239C29C75995A2C
:0646200022C29C7599FF07
:014626002271
:10307500E49002B5F0A3F0900383E0FFB4021A9048
:103085000A01E064A56006E4900383F022E490035E
:1030950084F0A3F0900382F022900A02E0FD7C0008
:1030A5002409FBEC33FA7E00C3EF9BEA6480F874D5
:1030B5008098505FED2407FDEC33FCD3EF9DEC6465
:1030C50080F87480985018900383E024FFF582E41B
:1030D5003409F583E0FF900384EE8FF012143390EA
:1030E5000383E0FFB40511900A04E064077003024E
:1030F50031DBE4900383F022EF640660030231DBE9
:10310500900A05E0640670030231DB900382E04417
:1031150020F022E4900383F0900A02E0FD2408F5F4
:1031250082E4340AF583E0FE74072DF582E4340A5F
:10313500F583E07C002400FFEC3EFE900384E06E06
:103145007003A3E06F6007900382E04480F0900372
:1031550082E0FF6006900A06F08007D25CE4900AE0
:1031650006F0E4900A02F0900A05740BF0900A0349
:10317500E0FFA3E0900A03F0A3EFF07F02900A02BC
:10318500E0FE2407FDE433FCEFC39DEC6480F87496
:103195008098501874002FF582E4340AF583E0FD19
:1031A5009002B5E48DF01214330F80D19002B5E092
:1031B500FCA3E0FF74072EF582E4340AF583EFF0F3
:1031C500ECFF900A02E02408F582E4340AF583EF67
:0631D500F0C29C75995A3E
:0131DB0022D1
:10480600900383E02400F582E4340AF583EFF09008
:104816000383E004F0E0C3948C4002E4F090038349
:10482600E064017027900A00E0FF54FEB59A10EF8D
:1048360020E006D259C25A8013D25AC259800D902E
:104846000A00E0645A6005E4900383F030590D9045
:104856000383E0640370301231DC802B305A2590DC
:104866000A02E02403FFE433FE900383E0D39FEEC5
:104876006480F8748098400F124580C25AE4900311
:1048860083F08003123075C25BE490038FF09003CF
:0748960090F0900380F02276
:1044D500900A00E0B45A06A3E064A56003305C448A
:1044E500900A02E02408FFE433FE900383E0C39FB3
:1044F500EE6480F87480984014D29CE4F0C2599020
:104505000A00F0A3F0A3F0A3F0D25B8060900383D0
:10451500E004F0C29CE02400F582E4340AF583E06F
:10452500F5998049900383E0FF6016900A02E02424
:1045350003FDE433FCC3EF9DEC6480F87480984080
:1045450017D29CE4900383F0C259900A00F0A3F0BF
:10455500A3F0A3F0D25B8015900383E004F0C29C26
:10456500E02400F582E4340AF583E0F599E490034C
:0B4575008FF0900390F0900380F02284
:1065F200900380E004F0C394044008E4F090038325
:04660200F0D29C2214
:10657F00304E119002B1E004F0C39405400BD24CA1
:0A658F007405F022E49002B1F0223E
:0E4376009002BDEFF0A3EDF0A3EAF0A3EBF090
:10438400C246E4A3F0304C03024420A3F09002BEE2
:10439400E0FF9002C2E0C39F40030244209002C1A8
:1043A400E0FF04F0EFC3940550429002BDE0FD7CB1
:1043B400009002F97401F0A3F09002BFE0FFA3E0C3
:1043C4009002FBCFF0A3EFF0E4FB7F36123324928C
:1043D40046304604801680C5E4F5C87F01125C1A95
:1043E4007F641261047F01125C1A80B19002C1E003
:1043F400C39405400480258015E49002C1F0900226
:10440400BDE004F09002BFE475F0011214337F01A3
:10441400125C1A9002C2E004F0024391A246B392E5
:034424004EA2465F
:014427002272
:0E4FD9009002C3EFF0A3EDF0A3EAF0A3EBF01B
:104FE700C246E4A3F0204C519002C7E0FF04F0EF63
:104FF700C3940550449002C3E0FD7C00A3E09002F7
:10500700EFF0A37401F09002C5E0FFA3E09002F176
:10501700CFF0A3EFF0E4FB7F361229B0924630467B
:1050270004801680C3E4F5C87F01125C1A7F6412FE
:1050370061047F01125C1A80AFA246B3924EA2466A
:015047002246
:106017007A027BA37D02E4FF124FD9502E9002A390
:10602700E07004A3E060249002A7E04480F07A02C5
:106037007BA77D017F041243769002A7E0547FF08F
:0C6047007A027BA77D017F0412437622C1
:104BEC00E49002A6F0A37450F0E4A3F0A374F8F0E0
:104BFC00E4A3F0A3F0A37470F0A37401F0A3740306
:104C0C00F0A374FFF0E4A3F03000199002A7E04485
:104C1C0008F09002ACE0FF9000CDE0540FFEEF4E98
:104C2C009002ACF030013E9002A7E04404F09002F8
:104C3C00ADE0FF9000CDE054F0FEEF4E9002ADF0F1
:104C4C009000CEE0FEA3E0FF7C007D32121684E4DF
:104C5C007B257A01F9F81214EFAD07AC06EC900243
:054C6C00AEF0A3EFF023
:014C71002220
:0F675C007A027BA67D0B7F031243769245A245FE
:01676B00220B
:106280007A027BA37D02E4FF124FD950259002A42D
:10629000E0FF30E102D24BEF30E002D24D9002A39A
:1062A000E030E304D215D2609002A4E030E20312A1
:0362B000675C2206
:106599007A027BB97D027F02124FD9500A9002B963
:0765A900E09002A5F0F526C9
:0165B00022C8
:105378009002BB7403F09002BBE0FFD3940B504C37
:105388007A027BB97D02124FD99002BBE0FF7E0002
:105398007B0124A3F9EE3402FA1213B3FD9002B98B
:1053A800E0B5051374A42FF9EE3402FA1213B3FF13
:1053B8009002BAE06F600C9002BBE06407600412D0
:0C53C800675C229002BBE02402F080AA87
:0153D40022B6
:1063EE009002B07433F07A027BB07D017F0D1243C0
:1063FE007650129002A7E04420F07A027BA77D012E
:06640E007F041243762218
:1065C8009002A8E054FCF04FF07A027BA87D017F8E
:0565D8000512437622CC
:106641009002A7E04401F07A027BA77D017F04124A
:036651004376226B
:106654009002A7E054FEF07A027BA77D017F04122A
:0366640043762258
:106667009002A7E04402F07A027BA77D017F041223
:0366770043762245
:10667A009002A7E054FDF07A027BA77D017F041205
:03668A0043762232
:105FD8009002BBEEF0A3EFF09002BBE0FEA3E078E6
:105FE80005CEC313CE13D8F99002AAF07A027BAA81
:105FF8007D017F0712437650159002BBE0A3E09025
:0F60080002ABF07A027BAB7D017F081243762258
:10668D009002A7E04410F07A027BA77D017F0412EF
:03669D004376221F
:1066A0009002A7E054EFF07A027BA77D017F0412ED
:0366B0004376220C
:1066B3009002A9E044F8F07A027BA97D017F0612DB
:0366C300437622F9
:1066C6009002A9E05407F07A027BA97D017F0612A9
:0366D600437622E6
:1066D9009002A9E044E0F07A027BA97D017F0612CD
:0366E900437622D3
:1066EC009002A9E0541FF07A027BA97D017F06126B
:0366FC00437622C0
:1066FF009002A9E04408F07A027BA97D017F06127F
:03670F00437622AC
:106712009002A9E054F7F07A027BA97D017F06126C
:0367220043762299
:10674A009002A6E04FF07A027BA67D017F031243F6
:02675A007622A5
:1065B1009002A6E0FEEFF4FFEE5FF07A027BA67D8B
:0765C100017F031243762263
:10346B003050030235AE3051030235AE2003030258
:10347B0035AEE490038AF0A3F0C3900063E095129D
:10348B00900062E09511500330181ED3900065E058
:10349B009512900064E09511400320180C20100940
:1034AB00201206201103301308C252E4900389F056
:1034BB0022C39000A4E095129000A3E09511400365
:1034CB000235A7C3E5129510FFE511950FFED390BA
:1034DB0000A6E09F9000A5E09E40030235A7900058
:1034EB00A7E0FEA3E0FFEE3395E0FDFC9002201277
:1034FB001609C312159C50030235A72052069003E0
:10350B0089E004F09000A9E075F00AA4FF9003890C
:10351B00E0C39FE5F06480F874809850030235AEE9
:10352B00AD14E5142513FFE433FEEDC39FEE648069
:10353B00F87480985063ED25E0240AF582E4340298
:10354B00F583E0FEA3E0C39510FFEE950FFED3903D
:10355B0000A6E09F9000A5E09E503BED25E0240ADD
:10356B00F582E43402F583E0FEA3E0FF9000A3E0D4
:10357B00FAA3E0FBC3EF9BEE9A401B74017E00A8FD
:10358B0005088005C333CE33CED8F9FF90038AE00C
:10359B004EF0A3E04FF00D8089D25222C252E4903C
:0335AB000389F0A1
:0135AE0022FA
:1061E200C24530052D20162A305427C39002B4E050
:1061F20094B49002B3E094005011D245900388E029
:1062020004F0C3940A400BD2168007C254E49003F0
:0462120088F0A24529
:016216002265
:10420900C3E5129510FFE511950FFEC3EF94B0EECB
:104219009404500AE5129464E51194055002D254AD
:10422900900386E024FE605514605914606A146096
:104239007C240460030242C220510330527B305374
:104249001590038AE05455FFA3E054559002B9CF65
:10425900F0A3EFF0801390038AE054AAFFA3E0547F
:10426900AA9002B9CFF0A3EFF09002B9E0FEA3E063
:10427900FF125FD89003867402F0D2502290038611
:104289007403F0221261E24030E4FFFE125FD8901D
:1042990003867404F0B253221261E2400790038648
:1042A9007405F0229003867401F0B25322900386BC
:0942B9007401F0C251C252C2505E
:0142C20022D9
:1064140030052220161F900387E004F0C3942D401A
:1064240014742DF020500EE4F0D25190038A7403BA
:06643400F0A374FFF0224A
:0A67940012346B1264141242092241
:10624C00FFD8FFE2FFECFFF60000000A0019002364
:10625C00002D00370041004B0055FFFBFFFCFFFDFC
:10626C00FFFEFFFFFFFF0000000100010002000322
:04627C000004000515
:0427C0008F828E83F3
:1027C4007E037FE8AD82AC83121684C006C007AED8
:1027D40083AF82C3E49FFF74109EFEAB07FAE4F953
:1027E400F8D007D0061214EF9002BC121615E47F3D
:1027F4000AFEFDFC9002BC121609D31215B2401D4C
:102804009002BC1215FDC3EF940AFFEE9400FEED96
:102814009400FDEC9400FC9002BC1216159035AFA8
:10282400E493FE740193FFE4FCFD9002BC121609CC
:10283400C31215B2400D9002BA7408F0A374B7F035
:102844000229A79036EFE493FE740193FFE4FCFDA4
:102854009002BC121609D31215B2500D9002BA742C
:102864000EF0A374F7F00229A790027CE09002B95D
:10287400F075F0029035AF121652E493FE74019392
:10288400FFE4FCFD9002BC121609D31215B2403BC2
:1028940090027CE0149002B9F09002B9E0FFC39476
:1028A40000406975F002EF9035AF121652E493FEC2
:1028B400740193FFE4FCFD9002BC121609D31215B7
:1028C400B240499002B9E014F080CE90027CE0045A
:1028D4009002B9F09002B9E0FFC394A0502875F0BB
:1028E40002EF9035AF121652E493FE740193FFE4A5
:1028F400FCFD9002BC121609D31215B250089002C6
:10290400B9E004F080CE9002B9E014F09002B9E08E
:1029140090027CF075F0029035AF121652E493FEEB
:10292400740193FFE4FCFD9002BC121609121456C4
:10293400E47B0AFAF9F8121464C004C005C006C0A6
:10294400079002B9E0FF75F0029035B1121652E417
:1029540093FC740193FD75F002EF9035AF1216529B
:10296400C37401939DFFE4939CFEAB07FAE4F9F86A
:10297400D007D006D005D0041214EFAB07AA0690F6
:10298400027CE024CEFFE434FFFE7C007D0A1213B7
:10299400CCEF2BFFEE3ACF24ABCF340A9002BAF03F
:0B29A400A3EFF09002BAE0FEA3E0FFFA
:0129AF002205
:105A6400D2459002C2E514F0E5132514FFE433FE99
:105A74009002C2E0C39FEE6480F87480985028E0DE
:105A8400FF25E02485F582E43402AB82FAEF25E0B9
:105A9400240EFF7D02124FD94005C245A245229033
:095AA40002C2E004F080C1A24539
:015AAD0022D6
:105BD200D2457A027B997D027F22124FD94002C2BE
:105BE200457A027B9B7D027F24124FD94002C24537
:105BF2007A027B9D7D027F26124FD94002C245E583
:105C020013D39405400F7A027B9F7D027F28124FA7
:075C1200D94002C245A24582
:015C19002268
:103A6200125BD24003023B4F900299E0FEA3E0FFBB
:103A72001227C09000D8E02FFF9000D7E03EFEC290
:103A8200AC900224F0A3EFF0D2AC90029DE0FEA332
:103A9200E0FFE4FCFD1212F47B9A7A9979D9783F1F
:103AA20012114EE4FBFA79F8784112105D121332CA
:103AB200C2AC900228EEF0A3EFF0D2ACE513D3949F
:103AC20005403290029FE0FEA3E0FFE4FCFD1212EB
:103AD200F47B9A7A9979D9783F12114EE4FBFA79FC
:103AE200F8784112105D121332C2AC90022AEEF045
:103AF200A3EFF0D2AC900224E0FCA3E0FD9002021E
:103B0200ECF0A3EDF0900204ECF0A3EDF0300D3DEB
:103B120090029BE0FEA3E0FF1227C09000DAE02FA4
:103B2200FF9000D9E03EFEC2AC900226F0A3EFF077
:103B3200D2ACD3900203E09F900202E09E4006EED8
:0D3B4200F0A3EFF022900204EEF0A3EFF0EC
:013B4F002253
:10382A009002BA121621000000009002BE12162160
:10383A0000000000E4900200F0A3F09002B37417B5
:10384A00F0A37470F0125A6440030239619002B90D
:10385A00E514F0E5132514FFE433FE9002B9E0FD08
:10386A00C39FEE6480F87480984003023938ED25CE
:10387A00E02485F582E43402F583E0FEA3E0FF7CD0
:10388A000E7DD8121684C006C0079000D1E0FEA3B0
:10389A00E0FFFBAA06E4F9F8D007D0061214EF906D
:1038AA0002BE121615900200E0FEA3E0FFE4FCFD42
:1038BA009002BE121609D31215B2400E9002BE1221
:1038CA0015FD900200EEF0A3EFF09002B3E0FEA324
:1038DA00E0FFE4FCFD9002BE121609C31215B250B5
:1038EA000E9002BE1215FD9002B3EEF0A3EFF02087
:1038FA005033C2AC9002BE1215FD9002B9E025E029
:10390A00240AF582E43402F583EEF0A3EFF0D2AC98
:10391A009002BA1215FD9002BE12160912144990AD
:10392A0002BA1216159002B9E004F002385D20506E
:10393A0026900200E0F511A3E0F5129002B3E0F53B
:10394A000FA3E0F510C2AC9002BA1215FD90021E48
:07395A00EEF0A3EFF0D2AC88
:013961002243
:1042C300E49002BEF0A3F0A3F09002C0E0FFC39419
:1042D3000C400302436DEF25E0244CF582E4346285
:1042E300F583E493FE740193FFFBAA06EA3395E09A
:1042F300F9F89002C0E025E0244EF582E43462F53B
:1043030083E493FE740193FFEE3395E0FDFC1214F6
:1043130049E47B02FAF9F8125E8FE47B0AFAF9F8B2
:10432300121464EF24ABFBEE340AFAE43DF9E43CE7
:10433300F8900228E0FEA3E0FFE4FCFDC312159C05
:10434300401F9002C0E025E02466F582E43462F564
:1043530083E493FF7401939002BECFF0A3EFF08048
:10436300099002C0E004F00242CC9002BEE0FEA33A
:02437300E0FF69
:014375002225
:102EFD009002BA121621000000007A027BA17D0219
:102F0D007F2A124FD99002A1E0FEA3E0FFEE30E43C
:102F1D000944E09002A1F0A3EFF01242C39000D556
:102F2D00E0FCA3E0FDC39002A2E09DFD9002A1E0B4
:102F3D009CCD2FFFED3EFE3395E0FDFC7B187AFC1A
:102F4D0079FF78FF121464C006C0079000D3E0FE2D
:102F5D00A3E0FFFBAA06EA3395E0F9F8D007D00607
:102F6D00125E8F90027D12161590027D1215FD9046
:102F7D0002B2E025E025E0243CF582E43402F5833D
:102F8D001216159002B2E004F0C394104002E4F062
:102F9D00E49002B9F09002B9E0FFC394105026A35B
:102FAD00121609EF25E025E0243CF582E43402F504
:102FBD00831215FD1214499002BA1216159002B91A
:102FCD00E004F080D0E47B10FAF9F89002BA121503
:102FDD00FD125E8F900281121615C22BC22A90002F
:102FED0028E0FEA3E0FFC3E49FFFE49EFE3395E0DF
:102FFD00FDFC900281121609C312159C50219003FD
:10300D009BE004F0C3940A405E740AF0D22BC2AC6C
:10301D009002811215FD900220121615D2AC22904D
:10302D000028E0FEA3E0FFEE3395E0FDFC90028169
:10303D00121609D312159C402090039AE004F094C7
:10304D000A4024740AF0D22AC2AC9002811215FDF6
:10305D00900220121615D2AC22C2AC90022012168C
:07306D002100000000D2ACBD
:013074002239
:10660600126280C24D12382A123A62304B05C24BD2
:04661600122EFD2221
:10504800E49002B9F0A3F0AF14E513FDE5142DFDCB
:10505800E433FCEFC39DEC6480F8748098501DEF36
:1050680025E02485F582E43402F583E0FCA3E0FD25
:105078009002B9EC8DF01214330F80CD9002B9E094
:10508800FEA3E0FF7C0E7DD8121684C006C00790F0
:105098000350E0FEA3E0FFFBAA06E4F9F8D007D02E
:0C50A800061214EF9000D1EEF0A3EFF020
:0150B40022D9
:10608E009000D5E0FEA3E0FFC39002A2E09FFF9038
:10609E0002A1E09EFE3395E0FDFC7B187AFC79FFB1
:1060AE0078FF121464900347121609125E8FEF4E9A
:0A60BE0060089000D3EEF0A3EFF0AD
:0160C80022B5
:10676C009002A1E0FFA3E09000D5CFF0A3EFF022C0
:105D7D00900299E0FEA3E0FF1227C0C390034DE00F
:105D8D009FFF90034CE09EFE9000D7E0FCA3E0FD4A
:105D9D00C3EF9DFDEE9CFCC3ED9496EC6480948066
:105DAD005012ED946AEC6480947F40089000D7EE19
:045DBD00F0A3EFF070
:015DC10022BF
:105DC20090029BE0FEA3E0FF1227C0C390034FE0C6
:105DD2009FFF90034EE09EFE9000D9E0FCA3E0FD01
:105DE200C3EF9DFDEE9CFCC3ED9496EC6480948021
:105DF2005012ED946AEC6480947F40089000D9EED2
:045E0200F0A3EFF02A
:015E06002279
:105E0700900352E0900378F0900353E0900379F009
:105E1700900354E090037AF0900355E090037BF0F1
:105E2700900356E090037CF0900357E090037DF0D9
:105E3700900358E090037EF07E037F7812476AD282
:045E47003BD23F22E9
:10583F0030734BC27390034BE030E003125048902B
:10584F00034BE030E40312608E90034BE030E5032E
:10585F0012676C90034BE030E203125D7D90034BB7
:10586F00E030E303125DC290034BE030E703125EBA
:0F587F0007E490034BF0D26A90039E7402F0226C
:1059CA0030600DC260D25EE490039DF012666722D9
:1059DA00305E3A126599203134900088E075F00201
:1059EA00A4FFAEF090039DE004F0C39FEE6480F83C
:1059FA007480984018C25EE4F012667A307002C26F
:0E5A0A0019C21BC21C301505C21512601722EE
:105E4B00305F0DC25FD25DE490039CF0126641227D
:105E5B00305D3012659920302A900088E075F00291
:105E6B00A4FFAEF090039CE004F0C39FEE6480F8B7
:105E7B00748098400EC25DE4F0126654306F02C21B
:045E8B0018C21A22FD
:10652900300719303C11900360E004F0C394054032
:0D6539000BD23A7405F022E4900360F022CA
:10525B009002E3EEF0A3EFF0A3EDF0A3EAF0A3EBE3
:01526B00F052
:10526C00C245203A41E4A3F09002E3E0FCA3E0FD48
:10527C00A3E09002F9F0E4A3F09002E6E0FFA3E0D3
:10528C009002FBCFF0A3EFF07B017FA012332450F0
:10529C0004D24580117F01125C1A9002E8E004F000
:0D52AC00E0C3940540C2A245B3923CA24568
:0152B90022D2
:1052BA009002C5EEF0A3EFF0A3EDF0A3EAF0A3EBA2
:0152CA00F0F3
:1052CB00C246203A41E4A3F09002C5E0FCA3E0FD06
:1052DB00A3E09002EFF0E4A3F09002C8E0FFA3E09C
:1052EB009002F1CFF0A3EFF07B017FA01229B05019
:1052FB0004D24680117F01125C1A9002CAE004F0BE
:0D530B00E0C3940540C2A246B3923CA24606
:015318002272
:1050B5007E027FBC7B08E4FD126376E49002BAF0C1
:1050C500A3F09002BAE0FEA3E0FFE4FCFD7BFF7ACB
:1050D50007F9F8D312159C402E53B1F89002BAE0A7
:1050E500FEA3E07805C333CE33CED8F9241FFFE401
:1050F5003EFE7A027BBC7D0112525B9002BAE475DA
:10510500F00112143380BB7A027BBC7D087FE07E00
:0B511500FF12525BE490035CF0A3F07B
:01512000226C
:104DF500C2457A027BB97D087FE07EFF1252BA92E6
:104E0500459002BAE0FF9002B9E02F9002BBF09006
:104E150002BEE0FF9002BDE02F9002BFF09002BC01
:104E2500E0FF9002BBE0B507179002B9E0FEA3E0F2
:104E35007C002400FFEC3E90035CF0A3EFF0802A99
:104E45009002C0E0FF9002BFE0B507179002BDE0F9
:104E5500FEA3E07C002400FFEC3E90035CF0A3EF92
:0C4E6500F08007E490035CF0A3F0A2458D
:014E7100221E
:105A1800E49002C3F07E037F78122B887E037F78A0
:105A28007C027DBA7B071262E6E4FF74BA2FF58226
:105A3800E43402F583E0FE9002C3E02EF00FEFB4E9
:105A480007E99002C3E09002C1F0A3745AF07A0209
:0B5A58007BBA7D097FF07EFF12525BDD
:015A63002220
:105F580090035CE0FCA3E0FDEC9002DBF0AF05A34E
:105F6800EFF09002DBE02F9002DEF09002DBE09091
:105F780002DFF09002DCE09002E0F09002DEE090B8
:105F880002E2F07A027BDB7D087FE07EFF12525B43
:015F980022E6
:052D4A009002BAEFF059
:102D4F006410701A7E037F617C027DBB7B0312626D
:102D5F00E67E037F657C027DBE1262E6801F7E03E6
:102D6F007F78122B887E037F787C027DBB7B0312DA
:102D7F0062E67E037F7B7C027DBE1262E6900206D6
:102D8F00E0FCA3E0FDEC9002C1F0A3EDF09002088F
:102D9F00E0FCA3E0FDEC9002C3F0A3EDF090022C59
:102DAF001215FD78181215C39002C5EFF090022C82
:102DBF001215FD78101215C39002C6EFF090022C79
:102DCF001215FD78081215C39002C7EFF090022C70
:102DDF001215FD9002C8EFF09002301215FD781811
:102DEF001215C39002C9EFF09002301215FD781042
:102DFF001215C39002CAEFF09002301215FD780839
:102E0F001215C39002CBEFF09002301215FD900215
:102E1F00CCEFF090021EE0FCA3E0FDAE047818CEDC
:102E2F00C313CE13D8F99002CDF0EDAE047810CEC7
:102E3F00C313CE13D8F99002CEF090021EE0FCA37C
:102E4F00E0FDEC9002CFF0A3EDF09002201215FD03
:102E5F0078181215D69002D1EFF09002201215FDBE
:102E6F0078101215D69002D2EFF09002201215FDB5
:102E7F0078081215D69002D3EFF09002201215FDAC
:102E8F009002D4EFF0900224E0FCA3E0FDEC90025E
:102E9F00D5F0A3EDF0900236E0FCA3E0FDEC90023C
:102EAF00D7F0A3EDF09002BAE09002D9F0A3745AD4
:102EBF00F090035CE0FEA3E0FF7A027BBB7D201263
:102ECF00525B90035CE475F02012143390035CE0C6
:102EDF00FEA3E0FFE4FCFD7BE07AFFF9F8D31215C7
:0D2EEF009C5007E490035CF0A3F0125F58C4
:012EFC0022B3
:10518C00900381E02480FFE434FFEF7D00C454F0F1
:10519C00FC900A01E02488FFE434FFFEEF7807C39B
:1051AC0033CE33CED8F92DFFEE3CFE900A02E0FD53
:1051BC007A0A7B031252BA7B017A0A7900900A02AE
:1051CC00E02403FD126563900A02E02403F582E4F7
:1051DC00340AF583EFF0C29C900383E02400F5823F
:0851EC00E4340AF583E0F599B3
:0151F4002298
:105CF2007E037F78122B887E037F787C0A7D037B6C
:105D0200071262E67B017A0A7900900A02E0240314
:105D1200FD126563900A02E02403F582E4340AF579
:105D220083EFF0C29C900383E02400F582E4340AFE
:065D3200F583E0F5992263
:10564C00300752303B4FC23B303905C2391250B58E
:10565C00303D05C23D12518C303805C238125CF217
:10566C00303F05C23F125A18303E0CC23E9002B970
:10567C007410F0FF122D4A30440CC2449002B974DD
:10568C0001F0FF122D4A30410CC2419002B9740254
:05569C00F0FF122D4A91
:0156A10022E6
:103B5000200703023C2290002EE0FF900359E0046E
:103B6000F0C39F4009E4F07E037F78122B88900316
:103B70005AE475F001121433FEC3E5F09410EE948C
:103B80000E400BE490035AF0A3F0D23BD23F202A20
:103B90001ED243304206C242D23BD24430190B30CF
:103BA0004008C240D23BD2418005201902D24030A9
:103BB000436990002CE0FEA3E0FFEE3395E0FDFCAE
:103BC000900220121609C312159C404F90035EE02C
:103BD0007002A3E070147E037F78122B887E037F2F
:103BE000787C037D617B071262E690002BE0FF7E0C
:103BF000007C007D3C1213CC90035EE475F0011252
:103C00001433FCD3E5F09FEC9E4017E490035EF084
:103C1000A3F0D242C243D23BD23E22E490035EF0F4
:033C2000A3F022EC
:0310530002512126
:10512100C0E0C0D075D000C006C007C0867586003B
:1051310030D807C2D87F0112648530D907C2D97F20
:105141000212648530DA07C2DA7F0412648530DB2B
:1051510007C2DB7F0812648530DC07C2DC7F1012D6
:10516100648530DD07C2DD7F2012648530DE07C231
:10517100DE7F4012648530DF07C2DF7F80126485E5
:0B518100D086D007D006D0D0D0E0329E
:03102B00021003AD
:10100300C0E0C083C082C0D0C086758640C28F75E1
:1010130086001264A9D086D0D0D082D083D0E032AB
:104627003074030246C875090F20A7057509018074
:104637000620B003750902E509650C6038050EE52B
:104647000E7002050DC3E50B940AE50A9400406558
:10465700E50E940AE50D94004067E50B9490E50A92
:1046670094014008E50C4440F5088003850C08D206
:104677007480428040E509640F6037E4F50DF50E5C
:10468700050BE50B7002050AB4900EE50AB40109A3
:10469700E50C4410F508D27422E50BB4B023E50A03
:1046A700B4041E750A01750B90E50C4420F508D279
:1046B700742275080FE4F50AF50BF50DF50E85095B
:0146C7000CE6
:0146C80022CF
:10621700AB07AA06C2AF43A701EAF5F7AF038FFBA7
:10622700AF058FFC75F26E75F30575F40A75F50900
:10623700EAADF7B50509E475F6060000000000535E
:05624700A7FED2AF220A
:10643A00D248E4FDFCEF2DFBEE3C8B82F583E4931E
:10644A006004C248800D0DBD00010CE4B505E6EC00
:05645A00B402E2A248BB
:01645F00221A
:0854E7009002BFEEF0A3EFF00C
:1054EF00D248AE04AF05E4A3F0A3F09002C1E0FCF4
:1054FF00A3E0FDC3EC940250369002C0E02DFD9066
:10550F0002BFE03C8D82F583E493FD9002C1E0FA87
:10551F00A3E02FF582EE3AF583E0FCED6C6004C258
:10552F0048800C9002C1E475F00112143380BCA2C4
:01553F004823
:015540002248
:084A52009002BFEEF0A3EFF0AB
:104A5A00C248AF05A3ECF0A3EFF0E4FDFC9002BF5F
:104A6A00E0FAA3E0FB2DF5FBEB2DEA3CF5F7A3E01A
:104A7A00FEA3E02DF582EE3CF583E0F5FC75F26EBF
:104A8A0020AF3D75F305E5A7603275F40A90039FE0
:104A9A00E06455702375F5099002C0E02D9002BFBD
:104AAA00E03CABF7B5030DE475F606000000000024
:104ABA00D2488010C2488019C2488015C248801165
:104ACA00C248800D0DBD00010CED7003EC6402704C
:034ADA008CA24863
:014ADD0022B6
:0E489D009002BBEEF0A3EFF0A3ECF0A3EDF061
:1048AB00C24753B1F8C2AF43A7019002BBE0FF7EF2
:1048BB0000F5F775F2E620AF5B75F305E5A76054DD
:1048CB0075F40A90039FE06455704975F509ADF7CF
:1048DB00EF6D7001EE703D75F60600000000009064
:1048EB0002BBE0FEA3E0FF12643A50289002BBE04B
:1048FB00FEA3E0FFA3E0FCA3E0FD124A525015908B
:10490B0002BBE0FEA3E0FFA3E0FCA3E0FD1254E733
:10491B005002D247E4F5F2F5F3F5F4F5F5F5F6535D
:08492B00A7FEF5F7D2AFA24789
:014933002261
:103C2300C245C246206903023CE3C26990039F7404
:103C330055F0E513D39405400C9002B97427F0A313
:103C43007410F0800A9002B97413F0A37488F09092
:103C530002B9E0FEA3E0FFC390021FE09F90021EA3
:103C6300E09E406B9001FEE0645A7004A3E064A5FB
:103C7300705DFDFCFFFE12489D4023E4FDFCFFFE4A
:103C830012489D4019D24574FF9001FEF0A3F0FD48
:103C93007FFE7E011262177DFF7FFF126217E4FD34
:103CA300FCFF7E0212489D402AE4FDFCFF7E0212C7
:103CB300489D401FD24674FF9001FEF0A3F0FD7FA4
:103CC300FE7E031262177DFF7FFF1262178004D20C
:103CD30045D246E490039FF0204505204602D26872
:013CE30022BE
:0E5319009002B9EEF0A3EFF0A3EAF0A3EBF0E0
:10532700D245AE04AF058E158F16C2AF43A7015302
:10533700B1F8E4FFFED39002BCE09F9002BBE09E71
:1053470040279002BAE02FFD9002B9E03E8D82F52A
:1053570083E493851682851583F00516E51670029A
:1053670005150FBF00010E80CC53A7FED2AFA24593
:015377002213
:1065DD00306A1190039EE004F0C394024006C26A33
:0565ED00E4F0D2692278
:1063A000C24543A701EEC313FEEF1325E0FFEE3312
:1063B0008F82F583740193B4A507E493B45A02D293
:0663C0004553A7FEA245B3
:0163C60022B4
:0D36F1009002BAECF0A3EDF09002B9EFF0FA
:1036FE00758640EF64557051A3E0FEA3E0FFC394BE
:10370E00E8EE940350187588027C007D2012168412
:10371E00C3E49FFFE49EA3F0A3EFF0023818758870
:10372E00229002BAE0FEA3E0FF7C007D20121684F8
:10373E00E47B40FAF9F81214EFC3E49FFFE49E9085
:10374E0002BCF0A3EFF00238189002B9E0644470A6
:10375E005BA3E0FEA3E0FFC394A0EE940F5023758D
:10376E0088127C007D80121684E47B08FAF9F81228
:10377E0014EFC3E49FFFE49E9002BCF0A3EFF002AF
:10378E0038187588329002BAE0FEA3E0FF7C007D07
:10379E0080121684E4FB7A01F9F81214EFC3E49F49
:1037AE00FFE49E9002BCF0A3EFF0805E9002B9E0C1
:1037BE007058A3E0FEA3E0FFC394F4EE94015022F0
:1037CE007588307C5D7DC0121684E4FB7A01F9F8B1
:1037DE001214EFC3E49FFFE49E9002BCF0A3EFF03F
:1037EE0080287588329002BAE0FEA3E0FF7C007D4F
:1037FE0080121684E4FB7A01F9F81214EFC3E49FE9
:10380E00FFE49E9002BCF0A3EFF09002BCE0FEA39A
:0B381E00E0F58CEEF58DD28AE4F58613
:01382900227C
:10579D00A2AFE433FEC2AFEF600D64206009EF6489
:1057AD00406004EFB46007EF4408F5B28010EF6479
:1057BD00806004EFB4A00753B2FB0053B2F70000B2
:1057CD00000000000000EF600D64206009EF6440F0
:1057DD006004EFB4600343B204AF06EE24FF92AF52
:0157ED002299
:104C7200900392EEF0A3EFF0A3EDF075C7B09003AE
:104C820092E0FEA3E0FFFBAA06E4F9F87FD87EB823
:104C92007D05FC125E8F8FCC900392E0FEA3E0FFB5
:104CA200FBAA06E4F9F87FD87EB87D05FC125E8F78
:104CB20078081215D68FCDAFCDEFFEADCC7C00E4D7
:104CC2002DFFEC3EFE900394E0FBFD1213CC7D64BD
:104CD2001213DE8FCEAFCDEFFEADCC7C00E42DFF04
:104CE200EC3EFEAD031213CC7D641213DEEEF5CF63
:014CF200229F
:104CF300900395EEF0A3EFF0A3EDF075B6B090033B
:104D030095E0FEA3E0FFFBAA06E4F9F87FD87EB89E
:104D13007D05FC125E8F8FAE900395E0FEA3E0FF4E
:104D2300FBAA06E4F9F87FD87EB87D05FC125E8FF6
:104D330078081215D68FAFAFAFEFFEADAE7C00E4AF
:104D43002DFFEC3EFE900397E0FBFD1213CC7D6438
:104D53001213DE8FA4AFAFEFFEADAE7C00E42DFFE8
:104D6300EC3EFEAD031213CC7D641213DEEEF5A50B
:014D7300221D
:104D74009002B9EEF0A3EFF0A3EDF075B7B0900296
:104D8400B9E0FEA3E0FFFBAA06E4F9F87FD87EB8F9
:104D94007D05FC125E8F8FBC9002B9E0FEA3E0FF9C
:104DA400FBAA06E4F9F87FD87EB87D05FC125E8F75
:104DB40078081215D68FBDAFBDEFFEADBC7C00E404
:104DC4002DFFEC3EFE9002BBE0FBFD1213CC7D6494
:104DD4001213DE8FBEAFBDEFFEADBC7C00E42DFF31
:104DE400EC3EFEAD031213CC7D641213DEEEF5BF70
:014DF400229C
:105C1A00E5B2547070067C067D868020E5B2547029
:105C2A00FEBE20067C037D438012E5B25470FEBEA0
:105C3A0040067C017DA180047C007D8BE4FEEEC3DE
:105C4A009F5014E4FBFAC3EB9DEA9C50070BBB0080
:075C5A00010A80F20E80E751
:015C61002220
:1062B3007F08AE07A806E4F60FEFD3949F40F3E4FC
:1062C300781EF608F6781EE6FE08E6FFD394FFEE86
:1062D300940A500E8F828E83E4F006E6187001064E
:0262E30080E356
:0162E5002296
:1051F50090002FE0645A705A900061E0645A705232
:10520500900074E0645A704A900089E0645A7042D4
:1052150090008EE0645A703A900099E0645A7032BA
:105225009000A2E0645A702A9000AAE0B45A239034
:1052350000CCE0B45A1C9000D0E0B45A159000DCC4
:10524500E0B45A0E9001FEE0645A7004A3E064A530
:065255006002C322D32217
:086376009002C5EEF0A3EFF068
:10637E00E4FFEFC39B501A9002C5E0F8A3E0F5824C
:10638E008883EDF09002C5E475F0011214330F808E
:01639E00E11D
:01639F0022DB
:0862E6009002DBEEF0A3EFF0E3
:1062EE00E4FFEFC39B50239002DBE0F8A3E0F582BE
:1062FE008883E08D828C83F00DBD00010C9002DB53
:0A630E00E475F0011214330F80D87B
:016318002262
:0C677C00758E55438701000000000022CC
:0C678800758E55438702000000000022BF
:10646000900391E06412701C305B19206A16206959
:1064700013C2AFF5A8F5A9F588F5E8F59DF59CF5EB
:0564800098120000224B
:105AAE00D228D229201403301602C22820110F202A
:105ABE00130C201B09201C06201503301602C229C8
:105ACE00202B0E201009201206201803301A02C2B5
:105ADE0028202A05301902C229201B06201C03305B
:0A5AEE001502C228301A02C2292254
:10634900125AAEA26D302801B34008A26E3029015D
:10635900B35019A228926DA229926EA229E433FFA3
:0D63690025E0FFA228E4334FFF1265C82293
:105C6200201844C3900063E09512900062E0951101
:105C7200501F900329E475F001121433FEC3E5F0BE
:105C82009401EE94004020D218E4900329F0A3F08E
:105C920022D3900065E09512900064E095114007D0
:085CA200E4900329F0A3F022B5
:105CAA00201944D3900076E09510900075E0950F86
:105CBA00401F90032BE475F001121433FEC3E5F084
:105CCA009401EE94004020D219E490032BF0A3F043
:105CDA0022C3900078E09510900077E0950F500766
:085CEA00E490032BF0A3F0226B
:10588E0020104B90008FE0FEA3E0FF900204E0FC9E
:10589E00A3E0FDD39FEC9E401F90033BE475F00107
:1058AE00121433FEC3E5F09401EE94004020D210A2
:1058BE00E490033BF0A3F022900091E0FEA3E0FF02
:0F58CE00C3ED9FEC9E5007E490033BF0A3F02244
:1058DD0020124B900093E0FEA3E0FF900202E0FC4B
:1058ED00A3E0FDC39FEC9E501F90033FE475F001B4
:1058FD00121433FEC3E5F09401EE94004020D21251
:10590D00E490033FF0A3F022900095E0FEA3E0FFAA
:0F591D00D3ED9FEC9E4007E490033FF0A3F022F0
:10592C0020114B90009AE0FEA3E0FF900204E0FCF3
:10593C00A3E0FDD39FEC9E401F90033DE475F00166
:10594C00121433FEC3E5F09401EE94004020D21102
:10595C00E490033DF0A3F02290009CE0FEA3E0FF56
:0F596C00C3ED9FEC9E5007E490033DF0A3F022A3
:10597B0020134B90009EE0FEA3E0FF900202E0FCA0
:10598B00A3E0FDC39FEC9E501F900341E475F00113
:10599B00121433FEC3E5F09401EE94004020D213B1
:1059AB00E4900341F0A3F0229000A0E0FEA3E0FFFF
:0F59BB00D3ED9FEC9E4007E4900341F0A3F02250
:1060C90030753712382A123A62125C62125CAA12CF
:1060D900588E1258DD12592C12597B9003A1E004F5
:1060E900F0C394024014C275204C09203A0620726C
:0B60F90003306803D2552212230F224F
:103DA100201859C3900063E09512900062E09511CC
:103DB1005033900066E075F00AA4FFAEF09003293D
:103DC100E475F001121433FCC3E5F09FEC9E50033F
:103DD100023E5CD218C26FE4900329F0A3F0900375
:103DE10043F0A3F022D3900065E09512900064E0C7
:103DF10095114067E4900329F0A3F022206F5CD372
:103E0100900065E09512900064E0951140379000B4
:103E110067E075F00AA4FFAEF0900343E475F0018A
:103E2100121433FCC3E5F09FEC9E402F300E06D2F6
:103E31006FD25F8002C218E4900329F0A3F09003CF
:103E410043F0A3F022C3900063E09512900062E07A
:0C3E510095115007E4900343F0A3F02209
:103E5D00201959D3900076E09510900075E0950FDC
:103E6D004033900079E075F00AA4FFAEF090032B7B
:103E7D00E475F001121433FCC3E5F09FEC9E500382
:103E8D00023F18D219C270E490032BF0A3F09003F7
:103E9D0045F0A3F022C3900078E09510900077E0F4
:103EAD00950F5067E490032BF0A3F02220705CC3B4
:103EBD00900078E09510900077E0950F50379000C6
:103ECD007AE075F00AA4FFAEF0900345E475F001B9
:103EDD00121433FCC3E5F09FEC9E402F300F06D239
:103EED0070D2608002C219E490032BF0A3F090030E
:103EFD0045F0A3F022D3900076E09510900075E088
:0C3F0D00950F4007E4900345F0A3F0225C
:103F190020105E90008FE0FEA3E0FF900204E0FC19
:103F2900A3E0FDD39FEC9E4031900097E075F0141B
:103F3900A4FFAEF090033BE475F001121433FAC309
:103F4900E5F09FEA9E5003023FD4D210E490033B70
:103F5900F0A3F090032DF0A3F022900091E0FEA3CE
:103F6900E0FFC3ED9FEC9E5062E490033BF0A3F0A9
:103F790022900091E0FEA3E0FF900204E0FCA3E0A0
:103F8900FDC39FEC9E502E900097E075F014A4FF9E
:103F9900AEF090032DE475F001121433FAC3E5F085
:103FA9009FEA9E4026C210E490033BF0A3F09003E1
:103FB9002DF0A3F02290008FE0FEA3E0FFD3ED9F48
:0C3FC900EC9E4007E490032DF0A3F022D2
:103FD50020125E900093E0FEA3E0FF900202E0FC59
:103FE500A3E0FDC39FEC9E5031900097E075F0145F
:103FF500A4FFAEF090033FE475F001121433FAC349
:10400500E5F09FEA9E5003024090D212E490033FF0
:10401500F0A3F0900331F0A3F022900095E0FEA309
:10402500E0FFD3ED9FEC9E4062E490033FF0A3F0E8
:1040350022900095E0FEA3E0FF900202E0FCA3E0E1
:10404500FDD39FEC9E402E900097E075F014A4FFE1
:10405500AEF0900331E475F001121433FAC3E5F0C4
:104065009FEA9E4026C212E490033FF0A3F090031E
:1040750031F0A3F022900093E0FEA3E0FFC3ED9F93
:0C408500EC9E5007E4900331F0A3F02201
:1040910020115E90009AE0FEA3E0FF900204E0FC94
:1040A100A3E0FDD39FEC9E4031900097E075F014A2
:1040B100A4FFAEF090033DE475F001121433FAC38E
:1040C100E5F09FEA9E500302414CD211E490033D7A
:1040D100F0A3F090032FF0A3F02290009CE0FEA348
:1040E100E0FFC3ED9FEC9E5062E490033DF0A3F02E
:1040F1002290009CE0FEA3E0FF900204E0FCA3E01C
:10410100FDC39FEC9E502E900097E075F014A4FF24
:10411100AEF090032FE475F001121433FAC3E5F009
:104121009FEA9E4026C211E490033DF0A3F0900364
:104131002FF0A3F02290009AE0FEA3E0FFD3ED9FC1
:0C414100EC9E4007E490032FF0A3F02256
:10414D0020135E90009EE0FEA3E0FF900202E0FCD3
:10415D00A3E0FDC39FEC9E5031900097E075F014E5
:10416D00A4FFAEF0900341E475F001121433FAC3CD
:10417D00E5F09FEA9E5003024208D213E4900341FA
:10418D00F0A3F0900333F0A3F0229000A0E0FEA383
:10419D00E0FFD3ED9FEC9E4062E4900341F0A3F06D
:1041AD00229000A0E0FEA3E0FF900202E0FCA3E05D
:1041BD00FDD39FEC9E402E900097E075F014A4FF68
:1041CD00AEF0900333E475F001121433FAC3E5F049
:1041DD009FEA9E4026C213E4900341F0A3F09003A2
:1041ED0033F0A3F02290009EE0FEA3E0FFC3ED9F0D
:0C41FD00EC9E5007E4900333F0A3F02286
:10554100201A5590006D1215FD90027D121609D397
:1055510012159C402A900071E075F00AA4FFAEF08C
:10556100900337E475F001121433FCC3E5F09FECAE
:105571009E4025D21AD25FE4900337F0A3F0222097
:105581005D16D3900338E09400900337E094004017
:095591000774FFF5F01214332237
:10559A00201B5590007E1215FD90027D121609C33C
:1055AA0012159C502A900082E075F00AA4FFAEF012
:1055BA00900325E475F001121433FCC3E5F09FEC67
:1055CA009E4025E4900325F0A3F0D21BD26022204E
:1055DA005E16D3900326E09400900325E0940040E1
:0955EA000774FFF5F012143322DE
:1055F300201C559000831215FD90027D121609C3DD
:1056030012159C502A900087E075F002A4FFAEF0BB
:10561300900327E475F001121433FCD3E5F09FECFB
:105623009E4025E4900327F0A3F0D21CD2602220F1
:105633005E16D3900328E09400900327E094004083
:095643000774FFF5F01214332284
:1064EC0020751B123DA1123E5D123F19123FD512B1
:0F64FC00409112414D12554112559A1255F322FB
:104F6300300272201B06201C03301539900072E0BA
:104F730075F014A4FFAEF0900339E475F001121438
:104F830033FCC3E5F09FEC9E401BE490039DF0903F
:104F93000339F0A3F0C21BC21CC260C25E30150508
:104FA300C215126017301A2D900072E075F014A428
:104FB300FFAEF0900335E475F001121433FCD3E532
:104FC300F09FEC9E400FE4900335F0A3F0C21A90DB
:064FD300039CF0C25D2208
:10654600300719307111900377E004F0C3940540C9
:0D6556000BD2727405F022E4900377F0225E
:0E5431009002F0EFF0A3EDF0A3EAF0A3EBF091
:10543F00C248207240E4A3F09002F0E0FD7C00A38C
:10544F00E09002F9F0E4A3F09002F2E0FFA3E09005
:10545F0002FBCFF0A3EFF0E4FB7FDE123324500406
:10546F00D24880117F01125C1A9002F4E004F0E040
:0C547F00C3940540C3A248B39271A24838
:01548B0022FE
:0E548C009002E6EFF0A3EDF0A3EAF0A3EBF040
:10549A00C247207240E4A3F09002E6E0FD7C00A33C
:1054AA00E09002EFF0E4A3F09002E8E0FFA3E090BE
:1054BA0002F1CFF0A3EFF0E4FB7FDE1229B0500433
:1054CA00D24780117F01125C1A9002EAE004F0E0F0
:0C54DA00C3940540C3A247B39271A247DF
:0154E60022A3
:082B88009002DBEEF0A3EFF078
:102B9000C2467A027BDD7D09E4FF12548C400302B9
:102BA0002D479002E4E030E003022D3A9002DFE08E
:102BB00020E703022C599002DDE0FF54709450404E
:102BC00003022C59EF540F94094003022C59E0548E
:102BD0007F94594003022C59A3E0FF547094505045
:102BE00078EF540F94095071E0547F9459506AA3C0
:102BF000E0FF543094205061EF540F9409505AE094
:102C0000542F94245053A3E0FF54309430504AEF93
:102C1000540F94095043E0543FFF9431503BEF6010
:102C200038A3E0FF54109410502FEF540F94095024
:102C300028E0541FFF94125020EF601DA3E0FF54C2
:102C4000F094905014EF540F9409500DE094995063
:102C500008A3E05407940640779002DBE0FEA3E06F
:102C6000FFF5828E83E09002DDF08F828E83A3E0F9
:102C70009002DEF09002DBE0A3E0F5828E83A3A356
:102C8000E09002DFF08F828E83A3A3A3E09002E0A6
:102C9000F09002DBE0A3E02404F582E43EF583E05B
:102CA0009002E1F0EF2405F582E43EF583E0900226
:102CB000E2F09002DBE0A3E02406F582E43EF58337
:102CC000E09002E3F07E027FDD12476A9246807751
:102CD0009002DDE0FF9002DBE0FCA3E0FDF5828CDA
:102CE00083EFF09002DEE08D828C83A3F09002DF10
:102CF000E0541F8D828C83A3A3F09002E0E08D82CC
:102D00008C83A3A3A3F09002E1E0FFED2404F582FD
:102D1000E43CF583EFF09002E2E0FFED2405F5825C
:102D2000E43CF583EFF09002E3E0FFED2406F5824A
:102D3000E43CF583EFF0D246800D9002DBE0FEA389
:092D4000E0FF12476A9246A24628
:012D49002267
:08476A009002E6EEF0A3EFF06F
:10477200C247A37490F07A027BE87D017F0712544E
:104782003192479002E6E0FEA3E0FFF5828E83E0DD
:104792009002E9F08F828E83A3E09002EAF0900209
:1047A200E6E0FCA3E0FDF5828C83A3A3E0448090C5
:1047B20002EBF08D828C83A3A3A3E09002ECF09035
:1047C20002E6E0A3E0FF2404F582E43EF583E090F4
:1047D20002EDF0EF2405F582E43EF583E09002EE6F
:1047E200F09002E6E0A3E02406F582E43EF583E0E1
:1047F2009002EFF07A027BE97D07E4FF12543192D6
:0348020047A24783
:014805002290
:0849C5009002B9EEF0A3EFF03F
:1049CD00C245E49002C4F07E027FBB7B09FD1263F9
:1049DD00767A027BBB7D097FF07EFF1252BAE4FF2F
:1049ED0074BB2FF582E43402F583E0FE9002C4E03F
:1049FD002EF00FEFB407E99002C4E0FF9002C2E081
:104A0D00B50706A3E0645A601BE49002BBF0A3F067
:104A1D00A37412F0A37401F0A37405F0A37420F035
:104A2D00A37405F07E027FBB9002B9E0FCA3E0FD0C
:104A3D007B071262E69002B9E0FEA3E0FF122B881D
:044A4D009245A245A7
:014A51002242
:1039620000070E091C1B1215383F363124232A2D5D
:1039720070777E796C6B6265484F464154535A5D4D
:10398200E0E7EEE9FCFBF2F5D8DFD6D1C4C3CACD3D
:1039920090979E998C8B8285A8AFA6A1B4B3BABD2D
:1039A200C7C0C9CEDBDCD5D2FFF8F1F6E3E4EDEA1D
:1039B200B7B0B9BEABACA5A28F88818693949D9A0D
:1039C2002720292E3B3C35321F18111603040D0AFD
:1039D2005750595E4B4C45426F68616673747D7AED
:1039E200898E878095929B9CB1B6BFB8ADAAA3A4DD
:1039F200F9FEF7F0E5E2EBECC1C6CFC8DDDAD3D4CD
:103A0200696E676075727B7C51565F584D4A4344BC
:103A1200191E171005020B0C21262F283D3A3334AC
:103A22004E49404752555C5B7671787F6A6D64639C
:103A32003E39303722252C2B0601080F1A1D14138C
:103A4200AEA9A0A7B2B5BCBB9691989F8A8D84837C
:103A5200DED9D0D7C2C5CCCBE6E1E8EFFAFDF4F36C
:10656300E4FFEDD3940040131213B36F9039629399
:0B657300FF740129F9E43AFA1D80E7EB
:01657E0022FA
:1063C700D24A7D807CBBE5C820E31053B1F8ED4C81
:1063D7006009ED1D70011C80ED80EBE5D154F86F6D
:0663E7006002C24AA24A56
:0163ED00228D
:103324009002F8EBF09002F5EFF0A3ECF0A3EDF0CF
:10333400D24990030174BBF0A37480F09002FDEFB6
:10334400F0A3EDF09002FBE0FEA3E0F5828E83E0B3
:103354009002FFF07B017A0279FD7D031265639090
:103364000300EFF09002F9E0D394005003023468B4
:1033740043E6C043D10143C80175C8607F081263A6
:10338400C7400C7F101263C74005C2490234459000
:1033940002F5E0F58D75C8407F181263C74005C279
:1033A400490234459002F8E0B401159002F6E0F5C4
:1033B4008D75C8407F281263C74005C24902344551
:1033C4009002F6E0A3E0F58D75C8407F281263C72C
:1033D4004004C249806B9002FAE06401702EA3E0BD
:1033E400FEA3E0F5828E83E0F58D75C8407F281238
:1033F40063C74004C2498049900300E0F58D75C855
:10340400407F281263C74039C2498035E4FE9002E8
:10341400F9E0FFEEC39F50299002FBE0FCA3E0F526
:10342400828C83E0F58D75C8407F281263C7400401
:10343400C249800D9002FBE475F0011214330E8032
:10344400CD75C850E5C830E41B53B1F8900301E0D2
:103454007002A3E0600E90030174FFF5F0121433C0
:0634640080E280E0A249B5
:01346A00223F
:0A29B000AA079002ECECF0A3EDF092
:1029BA00D248E4900322F0A374BBF0A37480F09091
:1029CA0002F4EAF0A3EDF09002EFE0FE9002F6F0D6
:1029DA00EA4401A3F0EED394005003022B8543E6A8
:1029EA00C043D10143C80175C8607F081263C7405C
:1029FA000C7F101263C74005C248022B628A8D758C
:102A0A00C8407F181263C74005C248022B62EBB464
:102A1A0001159002ECE0F58D75C8407F281263C756
:102A2A004005C248022B629002ECE0A3E0F58D75E6
:102A3A00C8407F281263C74005C248022B62EAB425
:102A4A0036159002EFE0F58D75C8407F281263C7EE
:102A5A004005C248022B6275C8607F081263C740EE
:102A6A000C7F101263C74005C248022B62EA440178
:102A7A00F58D75C8407F401263C74005C248022BD6
:102A8A0062E49002F3F09002EFE0FF9002F3E0FEBE
:102A9A00C39F50579002F0E07031EF14B5060A75E3
:102AAA00C8407F581263C7800875C8447F501263B4
:102ABA00C79002F1E0FEA3E0F5828E83E58DF090E7
:102ACA0002F1E475F001121433801875C8447F507E
:102ADA001263C79002F3E024F8F582E43402F58326
:102AEA00E58DF09002F3E004F0809B9002F0E06440
:102AFA0001706575C8407F581263C7900322E58D3F
:102B0A00F07B017A0279F49002EFE02404FD126569
:102B1A0063900322E0B5073EE49002F3F09002EFDF
:102B2A00E0FF9002F3E0FEC39F502D74F82EF58269
:102B3A00E43402F583E0FF9002F1E0FCA3E0F582C1
:102B4A008C83EFF09002F1E475F0011214339002D5
:102B5A00F3E004F080C7C24875C850E5C830E41BEA
:102B6A0053B1F8900323E07002A3E0600E900323B0
:0D2B7A0074FFF5F012143380E280E0A248F1
:012B8700222B
:1061040075C632E4F5E6EFFD7C007E5D7FC01213B8
:10611400DEEF24F0FFEE34FFC313FEEF13FFEEC4F3
:10612400F854F0C868EFC4540F48F58A75D1027565
:09613400C8407589FFE4F58D22D5
:084934009002B9EEF0A3EFF0D0
:10493C0075C432E4F587759850AB07AA06F9F87F71
:10494C00607EE37D16FC125E8FC3E49FFF74809E35
:10495C00AD07FCF59D8F9CFEAB07FAE4C39BFF747F
:10496C00809AFEE49400FDE49400FCE47B10FAF9D8
:10497C00F8121464EC1212F4C004C005C006C0078F
:10498C009002B9E0FCA3E0FDE41212F9A804A90519
:10499C00AA06AB077F007E1B7DB77C4B121257D04B
:1049AC0003D002D001D0001210591213328F9E4343
:0849BC009D80759A0A759BFFAE
:0149C40022D0
:031023000257EE83
:1057EE00C0E0C0F0C083C082C0D075D000C000C081
:0D57FE0001C002C003C004C005C006C00702
:10580B00C086758600309807C298AF99124806304B
:09581B009905C2991244D5D0860A
:10582400D007D006D005D004D003D002D001D000D8
:0B583400D0D0D082D083D0F0D0E03282
:1035AF00FFFFFFFFF07FDFCDD0DAC222B4F4A8C255
:1035BF009D769300894E804F77F770386906625673
:1035CF005C1F565650F44BF1474642EC3EDD3B1420
:1035DF003728343F312A2E462B97291226B62481BD
:1035EF002270207F1EAE1CFA1B6119E11878172676
:1035FF0015E714BC13A2129911A010B50FD80F081C
:10360F000E440D8A0CDC0C370B9C0B090A7E09FB50
:10361F00097E090A089B083207CF0770071706C3F0
:10362F000673062705DF059B055A051D04E204AB4B
:10363F0004770445041503E803BC0393036C0346A6
:10364F000325030302E302C502A8028C027102588C
:10365F0002400229021301FE01EA01D701C501B39D
:10366F0001A301930183017501670159014D0140C8
:10367F0001350129011F0114010A010100F800EFB2
:10368F0000E600DE00D700CF00C800C100BA00B4CA
:10369F0000AE00A800A2009D00980092008E008945
:1036AF0000840080007C007800740070006D006959
:1036BF00006600630060005D005A0057005400521E
:1036CF00004F004D004A00480046004400420040B1
:1036DF00003E003C003B0039003700360035003417
:0236EF000032A7
:0310000002661A6B
:10661A0075819F75B208000000000000000043B2B7
:04662A0004024EEB2D
:10230F007F647E00C262E4781BF608F67817F60841
:10231F00F608F608F6781DF6900373F0A3F0900315
:10232F006CF0A3F0900370F0A3F0A3F090036EF0A5
:10233F00900375F0A3F0C263C2619002B9F09002EE
:10234F00B9E0FDC3940A4003022452ED25E02402B4
:10235F00F582E43400F583E0FCA3E0D39512EC950D
:10236F001150030224499002B9E070529000B1E07D
:10237F00FCA3E0FDD39512EC95115003301906E440
:10238F00FEFF022452C3E5129DFFE5119CFE7C0067
:10239F007D0A121684C006C0079000B1E0FEA3E0CC
:1023AF00FFC3900003E09FFF900002E09EFEAB078B
:1023BF00FAE4F9F8D007D0061214EF022452900273
:1023CF00B9E025E02400F582E43400F583E0FEA3B4
:1023DF00E0FFC3E5129FFFE5119EFE7C007D0A1210
:1023EF001684C004C005C006C0079002B9E0FF25DF
:1023FF00E02400F582E43400F583E0FCA3E0FDEF78
:10240F0025E02402F582E43400F583E0FEA3E0C367
:10241F009DFFEE9CFEAB07FAE4F9F8D007D006D08B
:10242F0005D0041214EFAD07AC069002B9E075F0B9
:10243F000AA42DFFE5F03CFE80099002B9E004F0FC
:10244F0002234DD3900011E09512900010E09511EA
:10245F0050047E007F649000B5E0FD7C00D3EF9DBB
:10246F00EE9C40067E00AF05801EC3ED9FFDEC9EE7
:10247F00FCD3ED941EEC940040079000B5EFF08074
:10248F00079000B5E0FF7E00900234EEF0A3EFF06E
:10249F009000BA1215FD90022C121615900234E01E
:1024AF00FEA3E0FFE4FCFD90022C12160912146447
:1024BF00E47B64FAF9F81214EF90023012161590BB
:1024CF00022C1215FD900373EEF0A3EFF090023083
:1024DF001215FD90036CEEF0A3EFF0900234E0FEC6
:1024EF00A3E0FF7C007D0A1213CC900370EEF0A3E3
:1024FF00EFF09000CAE0FEA3E0FFD394C8EE940083
:10250F004006781D764B803DD3EF9464EE940040E7
:10251F00107C007D051213DEC3745F9F781DF6805B
:10252F00249000CAE0FEA3E0FFD39432EE94004063
:10253F00107C007D0A1213DEC374699F781DF6802C
:10254F0004781D7664E47819F608F6900372F0901B
:0B255F000375F0A3F0C26290036EF061
:01256A00224E
:101FE900E49002B9F0A3F0900368121621000000F2
:101FF90000900028E0FEA3E0FFEE3395E0FDFC90A1
:102009000220121609D312159C500302216FE49085
:102019000372F0900375F0A3F0C262781DE6FFE445
:10202900FCFDFE9000BE121609121464E47B64FAEA
:10203900F9F81214EF9002B9EEF0A3EFF0900373E0
:10204900E06E7003A3E06F602F900234E0FCA3E020
:10205900FD9002B9E0FEA3E0FF1213CC7C007D6481
:102069001213DE90036CEEF0A3EFF0C2ACE4FCFDBA
:10207900900230121615D2AC9002B9E0FFA3E0909D
:102089000373CFF0A3EFF09002811215FD781CEFD6
:1020990026F618EE36F6C3781CE6941018E6940E68
:1020A90040380874F026F61874F136F6900373E098
:1020B900FEA3E0FFC390036DE09F90036CE09E5088
:1020C90009E475F00112143380CC90036CEEF0A38F
:1020D900EFF0E4781BF608F680BC900373E0FEA3EA
:1020E900E0FF90036CE0FCA3E0FDC39FEC9E502A47
:1020F9007E037FE8121684C006C007900373E0FED2
:10210900A3E0FFFBAA06E4F9F8D007D0061214EF02
:10211900900370EEF0A3EFF0800A9003707403F05F
:10212900A374E8F09000ADE0FEA3E0FFEE3395E084
:10213900FDFC900281121609C312159C5022C3900E
:1021490000ACE095129000ABE0951150139000AFF0
:10215900E0FF90036EE004F0C39F4004EFF0D26407
:1021690012256B022240900028E0FEA3E0FFC3E4A1
:102179009FFFE49EFE3395E0FDFC900220121609B4
:10218900C312159C4003022240E490036EF0C2641E
:102199009002811215FD90036812161590036812BA
:1021A90015FDEC33500AC37818E69FF618E69EF63B
:1021B900C37818E6941018E6940E4078C37818E6A8
:1021C900941018E6940E403B0874F026F61874F142
:1021D90036F69000C61215FDEF2401FFE43EFEE439
:1021E9003DFDE43CFC9000C6121615D390036DE04A
:1021F900940190036CE0940040C274FFF5F012144E
:102209003380B99000C21215FD9000C6121609C399
:102219001215B2401F9000C61215FD9000C2121689
:10222900091214569000C61216159000CAE475F0EA
:1022390001121433121B8B301832C2AC900373E0B5
:10224900FEA3E0FF90036CEEF0A3EFF0E4FCFD9039
:1022590002301216159002301215FD90022C12163A
:1022690015900234E4F0A37464F0D2AC900373E0E7
:10227900FEA3E0FF90036CE0FAA3E0FBD39FEA9E84
:10228900400A90036CEEF0A3EFF0801DEF25E0FF0C
:10229900EE33FE7C007D641213DEC3EB9FEA9E5091
:1022A9000890036CEEF0A3EFF090036CE0FEA3E05E
:1022B900FF7C037DE8121684C006C007900373E013
:1022C900FEA3E0FFFBAA06E4F9F8D007D006121432
:1022D900EF900370EEF0A3EFF01216B1C2AC9002CA
:1022E90034E0A3E09000B5F090022C1215FD9000A7
:1022F900BA1216159000CAE0FFA3E0900236CFF09B
:05230900A3EFF0D2ACCF
:01230E0022AC
:10256B00E49002BBF09002BBE0FFC394095020EF54
:10257B0025E02402F582E43400F583E0FEA3E0C3FA
:10258B009512EE951150089002BBE004F080D63006
:10259B006458C3900371E094E7900370E094035088
:1025AB004990036DE004F0700690036CE004F0902A
:1025BB00036CE0FEA3E0FFE4FCFDEEC0E0EFC0E047
:1025CB00900373E0FEA3E0FFFBCAEECAE4F9F8D078
:1025DB00E0FFD0E0FE1214EFE47BE87A03F9F81287
:1025EB001464900370EEF0A3EFF09002BBE0701A4E
:1025FB00D39000B2E095129000B1E0951150030218
:10260B0027BFE4900234F0A3F022900014E0FEA365
:10261B00E0FFC39512EE951140030226BF9000AC6C
:10262B00E095129000ABE0951150030226BF306489
:10263B00030226BF900371E09484900370E094032F
:10264B0040030227BFC3E5129FFFE5119EFE7C00EE
:10265B007D64121684EEC0E0EFC0E0900014E0FE43
:10266B00A3E0FFC39000ACE09FFF9000ABE09EFEA9
:10267B00CBEFCBFAE4F9F8D0E0FFD0E0FE1214EF89
:10268B00EF2484FFEE3403900370F0A3EFF090037C
:10269B0073E0FEA3E0FF900370E0FCA3E0FD1216D5
:1026AB0084E47BE87A03F9F81214EF90036CEEF0F4
:1026BB00A3EFF0223064030227BF9002BBE0F97551
:1026CB00F064A42432FFE435F0FE900370E0FCA329
:1026DB00E0FDD39FEC9E5011E975F064A4FFC3EDB0
:1026EB009FEC95F040030227BF9002BBE0FF25E073
:1026FB002400F582E43400F583E0FCA3E0FDEF2534
:10270B00E02402F582E43400F583E0FEA3E06D7073
:10271B0002EE6C70030227BFC3E5129DFFE5119C0F
:10272B00FE7C007D64121684ECC0E0EDC0E0EEC0D0
:10273B00E0EFC0E09002BBE0FF25E02400F582E46F
:10274B003400F583E0FCA3E0FDEF25E02402F582E5
:10275B00E43400F583E0FEA3E0C39DFFEE9CFECBCB
:10276B00EFCBFAE4F9F8D0E0FFD0E0FED0E0FDD0FB
:10277B00E0FC1214EFCDEFCDCCEECC9002BBE075AC
:10278B00F064A42DFEE5F03C900370F0A3CEF09026
:10279B000373E0FEA3E0FF900370E0FCA3E0FD12E7
:1027AB001684E47BE87A03F9F81214EF90036CEECD
:0427BB00F0A3EFF0A8
:0127BF0022F7
:101B8B00E49002BBF0A3F0A3F0A3F0A3F0A3F0A3A7
:101B9B00F0A3F0A3F07819E6FE08E6FF2414FDE4A9
:101BAB003EFC900204E0FAA3E0FBD39DEA9C5011AB
:101BBB00EB2414FDE43AFCD3EF9DEE9C5003021D85
:101BCB0092900204E0FEA3E0FF7819EEF608EFF620
:101BDB002487FFEE34F5FE9002BDF0A3EFF07C00FE
:101BEB007D111213CCC374689FFF74429EFECBEF22
:101BFB00CBFA3395E0F9F89002BDE0FEA3E0FFEEDF
:101C0B003395E0FDFC121464E47B107A27F9F8128B
:101C1B005E8FEF2422FFEE3406FEE43DFDE43CFC38
:101C2B009000B6E0F8A3E0F9A3E0FAA3E0FB1214EE
:101C3B0064E47BD07A07F9F81214EF9002C2EEF04D
:101C4B00A3EFF0E4FCFD9000B6E0F8A3E0F9A3E00D
:101C5B00FAA3E0FBC31215B250159000B6E0A3E057
:101C6B00A3E0FFA3E09002C2CFF0A3EFF08065E406
:101C7B007F06FEFDFC9000B6E0F8A3E0F9A3E0FAC6
:101C8B00A3E0FB121464E47B0AFAF9F81214EFC810
:101C9B00ECC8C9EDC9CAEECACBEFCB9002C2E0FECD
:101CAB00A3E0FFE4FCFDD31215B24028E47F06FE4F
:101CBB00FDFC9000B6E0F8A3E0F9A3E0FAA3E0FB8B
:101CCB00121464E47B0AFAF9F81214EF9002C2EED4
:101CDB00F0A3EFF09002C2E0FEA3E0FF781DE6FD5B
:101CEB007C00121684E47B64FAF9F81214EF90026C
:101CFB00C2EEF0A3EFF0900373E0FCA3E0FDD39FE3
:101D0B00EC9E501BC39002C3E09DFF9002C2E09C6F
:101D1B00FE90036DE02FF090036CE03EF0804A9054
:101D2B0002C2E0FEA3E0FFC3900374E09FFF9003A9
:101D3B0073E09EFEC390036DE09F90036CE09E40AA
:101D4B000CA3E09FF090036CE09EF0801C9002C20D
:101D5B00E0FEA3E0FF7C007D061213CC7D64121322
:101D6B00DE90036CEEF0A3EFF0C39000B2E09510A1
:101D7B009000B1E0950F500F9002C2E0FFA3E090EE
:101D8B000373CFF0A3EFF0D3900205E094DD900244
:101D9B0004E0940A5003021FE874FF7FFAFEFDFC77
:101DAB009000B6E0F8A3E0F9A3E0FAA3E0FB12146D
:101DBB0064C8ECC8C9EDC9CAEECACBEFCB90022000
:101DCB00E0FCA3E0FDA3E0FEA3E0FFC31215B240CD
:101DDB0003021FE8900373E0FEA3E0FF7C007D0687
:101DEB001213CC7D641213DE9002BBEEF0A3EFF066
:101DFB00900368E0FCA3E0FDA3E0FEA3E0FF126705
:101E0B009EE47B0AFAF9F81214649000B6E0F8A38A
:101E1B00E0F9A3E0FAA3E0FB1214EF9002BFEFF09E
:101E2B00E47F19FEFDFC900368E0F8A3E0F9A3E062
:101E3B00FAA3E0FB121464E47BE87A03F9F8125E70
:101E4B008FEF2416FFEE340D9002C0F0A3EFF0C31A
:101E5B009000B2E095109000B1E0950F50429002C7
:101E6B00BBE0FEA3E0FFC390036DE09F90036CE02B
:101E7B009E502DC3900371E0942C900370E094015D
:101E8B00501E20621B9000B0E0FF900375E004F041
:101E9B00C39F5003021F93EFF0D263C261021F93E3
:101EAB009002C0E0FEA3E0FFC39510EE950F5042E9
:101EBB009002BBE0FCA3E0FDC390036DE09D90039B
:101ECB006CE09C502DC3900371E0942C900370E058
:101EDB009401501E20621B9000B0E0FD900375E052
:101EEB0004F0C39D5003021F93EDF0D263C2610255
:101EFB001F93D3EF9510EE950F403D9002BBE0FE84
:101F0B00A3E0FFD390036DE09F90036CE09E40280D
:101F1B00900371E0942C900370E09401501A2062AE
:101F2B00179000B0E0FF900376E004F0C39F405899
:101F3B00EFF0C263D2618050D39000B2E095109065
:101F4B0000B1E0950F403D9002BBE0FEA3E0FFD354
:101F5B0090036DE09F90036CE09E4028900371E02E
:101F6B00942C900370E09401501A2062179000B0EB
:101F7B00E0FF900376E004F0C39F400CEFF0C263E8
:101F8B00D2618004C263C261C39000B2E09510902D
:101F9B0000B1E0950F40469000B0E0FF900372E077
:101FAB0004F09F4038EFF0D2629002BFE0941E50D5
:101FBB001D900374E025E0FF900373E033FE7C007B
:101FCB007D641213DE90036CEEF0A3EFF02290020F
:0D1FDB00BBE0FFA3E090036CCFF0A3EFF09C
:011FE80022D6
:1016B1009002BC121621000000009002C0121621F7
:1016C10000000000900370E0FEA3E0FF7C007D0AB3
:1016D1001213DE9002BBEFF0900220E0FCA3E0FDCC
:1016E100A3E0FEA3E0FFEC4D4E4F7003021B63909D
:1016F10002BBE0FFC3900235E09F900234E094000A
:101701004003021871E4FFFEFDFC900220E0F8A303
:10171100E0F9A3E0FAA3E0FB12159C500302187153
:101721009002BBE0FF900234E0FCA3E0FDEF9DFFDF
:10173100E49CFEC3EF9401EE9400500302183F7C39
:10174100007D64121684E47B1EFAF9F81214EF90FE
:1017510002BC1216159002BCE0FCA3E0FDA3E0FE62
:10176100A3E0FF90022CE0F8A3E0F9A3E0FAA3E0E4
:10177100FB121464E47B107A27F9F81214EF90023B
:10178100C0121615900230E0FCA3E0FDA3E0FEA319
:10179100E0FF9002C0E0F8A3E0F9A3E0FAA3E0FBC8
:1017A100EF2BFFEE3AFEED39FDEC38FC90023012E2
:1017B1001615900373E0FEA3E0FFE4FCFD90022CFC
:1017C100121615E47F64FEFDFC900230E0F8A3E000
:1017D100F9A3E0FAA3E0FB12146490022CE0F8A351
:1017E100E0F9A3E0FAA3E0FB1214EFC8ECC8C9EDDD
:1017F100C9CAEECACBEFCB900234E0FEA3E0FFE40E
:10180100FCFDC31215B25003021B63E47F64FEFDAD
:10181100FC900230E0F8A3E0F9A3E0FAA3E0FB12A8
:10182100146490022CE0F8A3E0F9A3E0FAA3E0FB32
:101831001214EF900234EEF0A3EFF0021B63900359
:1018410073E0FEA3E0FFE4FCFD90022C121615905C
:10185100036CE0FEA3E0FFE4FCFD900230121615DC
:101861009002BBE0FF900234E4F0A3EFF0021B63AF
:101871009002BBE0F9FF900234E0FAA3E0FBD39FB2
:10188100EA94005003021AE9900220E0FCA3E0FD73
:10189100A3E0FEA3E0FFEC334003021AE9E9FFEB0A
:1018A1006F7001EA703220632F20612C900373E086
:1018B100FEA3E0FFE4FCFD90022C12161590036CD0
:1018C100E0FEA3E0FFE4FCFD900230121615E9FFF3
:1018D100900234E4F0A3EFF0900234E0FEA3E0FFC5
:1018E100D39401EE94005003021AAB900076E024E9
:1018F10064FD900075E03400FCD3E5109DE50F9C7C
:101901005003021A98EF940FEE94004003021A98C4
:10191100206306206103021A9874FF7FFDFEFDFC1F
:101921009000B6E0F8A3E0F9A3E0FAA3E0FB1214FB
:1019310064C8ECC8C9EDC9CAEECACBEFCB9002208E
:10194100E0FCA3E0FDA3E0FEA3E0FFD31215B2404B
:1019510035900220E0FCA3E0FDA3E0FEA3E0FF122E
:10196100158EE47B02FAF9F81214649000B6E0F8DF
:10197100A3E0F9A3E0FAA3E0FB1214EF9002C5EE95
:10198100F0A3EFF080089002C5E4F0A304F090000A
:1019910075E0FEA3E0FFC39510EE950F5017C3E568
:1019A100109FFFE50F9EFE7C007D821213DE9002E8
:1019B100C4EFF080069002C47401F09000B6E0FC20
:1019C100A3E0FDA3E0FEA3E0FF12158EE47B24FA61
:1019D100F9F8121464ECC0E0EDC0E0EEC0E0EFC035
:1019E100E0900220E0FCA3E0FDA3E0FEA3E0FFFB0A
:1019F100CAEECAC9EDC9C8ECC8D0E0FFD0E0FED03C
:101A0100E0FDD0E0FC1214EFCDEFCDCCEECC900296
:101A110034E0A3E0FF9002BBE0FEC3EF9E04FB9025
:101A210002C4E0FF7E001213CCCDEBCD7C0012137B
:101A3100DEA3E0FCA3E0FD1213DE90036FE004F0EF
:101A4100D39FE49E4013900235E024FFF0900234CE
:101A5100E034FFF0E490036FF0900234E0FEA3E085
:101A6100FF7C007D0A1213CC900370EEF0A3EFF01F
:101A7100900373E0FEA3E0FF900370E0FCA3E0FDA0
:101A8100121684E47BE87A03F9F81214EF90036CE0
:101A9100EEF0A3EFF08013900235E024FFF0900206
:101AA10034E034FFF0E490036FF0900373E0FEA3A1
:101AB100E0FFE4FCFD90022C121615900234E0FECA
:101AC100A3E0FFE4FCFD90022CE0F8A3E0F9A3E021
:101AD100FAA3E0FB121464E47B64FAF9F81214EF40
:101AE100900230121615807A9002BBE0FB7A0090CA
:101AF1000234E07003A3E06B702C900373E0FEA34B
:101B0100E0FFE4FCFD90022C12161590036CE0FE40
:101B1100A3E0FFE4FCFD900230121615900234EAB6
:101B2100F0A3EBF0803C900373E0FEA3E0FFE4FC44
:101B3100FD90022C121615900234E0FEA3E0FFE4A2
:101B4100FCFD90022CE0F8A3E0F9A3E0FAA3E0FB8E
:101B5100121464E47B64FAF9F81214EF9002301263
:101B61001615900234E0FEA3E0FFD39464EE9400D6
:101B7100400A900234E4F0A37464F022C3EE9400AE
:091B81005007E4900234F0A3F0D7
:011B8A002238
:10672500305C0F305B0CC25CC25BC2AF1266A0125C
:0367350000A62299
:108400002B370C800D480DDE0E740ED80F3C0FA0DC
:10841000100410361068000008980000089800004A
:10842000083400000AAB00C8006414010064055A57
:10843000021101200053696E6F7765616C746800EA
:1084400000202206200000534833394630303400E3
:108450000000004C494F4E000000000000000000EA
:10846000005A109A10360202000000000000000BB3
:10847000B8020A005A0A8C0BB80202000000FFFF83
:10848000B1E002FFFF63C002045A0FA01E465A0C5F
:108490009F0C6D0AAB0ADD03035A0D670CD10A4726
:1084A0000A795A105400140064025A1068006405D6
:1084B000050B540AAB6400000898000008980000FF
:1084C0000898000008340000000000005A741130C1
:1084D0005A0A22FFAE000100000000005A0000000E
:1084E000000000000000000000000000000000008C
:1084F000000000000000000000000000000000007C
:10850000000000000000000000000000000000006B
:10851000000000000000000000000000000000005B
:10852000000000000000000000000000000000004B
:10853000000000000000000000000000000000003B
:10854000000000000000000000000000000000002B
:10855000000000000000000000000000000000001B
:10856000000000000000000000000000000000000B
:1085700000000000000000000000000000000000FB
:1085800000000000000000000000000000000000EB
:1085900000000000000000000000000000000000DB
:1085A00000000000000000000000000000000000CB
:1085B00000000000000000000000000000000000BB
:1085C00000000000000000000000000000000000AB
:1085D000000000000000000000000000000000009B
:1085E000000000000000000000000000000000008B
:1085F00000000000000000000000000000005AA57C
:108600002B370C800D480DDE0E740ED80F3C0FA0DA
:108610001004103610680000089800000898000048
:10862000083400000AAB00C8006414010064055A55
:10863000021101200053696E6F7765616C746800E8
:1086400000202206200000534833394630303400E1
:108650000000004C494F4E000000000000000000E8
:10866000005A109A10360202000000000000000BB1
:10867000B8020A005A0A8C0BB80202000000FFFF81
:10868000B1E002FFFF63C002045A0FA01E465A0C5D
:108690009F0C6D0AAB0ADD03035A0D670CD10A4724
:1086A0000A795A105400140064025A1068006405D4
:1086B000050B540AAB6400000898000008980000FD
:1086C0000898000008340000000000005A741130BF
:1086D0005A0A22FFAE000100000000005A0000000C
:1086E000000000000000000000000000000000008A
:1086F000000000000000000000000000000000007A
:108700000000000000000000000000000000000069
:108710000000000000000000000000000000000059
:108720000000000000000000000000000000000049
:108730000000000000000000000000000000000039
:108740000000000000000000000000000000000029
:108750000000000000000000000000000000000019
:108760000000000000000000000000000000000009
:1087700000000000000000000000000000000000F9
:1087800000000000000000000000000000000000E9
:1087900000000000000000000000000000000000D9
:1087A00000000000000000000000000000000000C9
:1087B00000000000000000000000000000000000B9
:1087C00000000000000000000000000000000000A9
:1087D0000000000000000000000000000000000099
:1087E0000000000000000000000000000000000089
:1087F00000000000000000000000000000005AA57A
:1010560002139EE86480F8E933E83360110460F017
:10106600ED33EC337009E8FCE9FDEAFEEBFF220400
:1010760060DED3EB9FEA9EE99DE8C2E78CF0C2F7FB
:1010860095F0400CE8CCF8E9CDF9EACEFAEBCFFBC7
:1010960012136985D0F05804700320D5B3E80470A4
:1010A600075002B2D50213A892D5EC0460F7E4CC3F
:1010B600C0E0C398F8603B94186008400DD0E0FB90
:1010C600021380E4FBFAC9FC8028E830E406E4C990
:1010D600FBE4CAFCE830E305E4C9CACBFCE85407E4
:1010E6006010F8C3E913F9EA13FAEB13FBEC13FCEF
:1010F600D8F130F52FC3E49CFCEF9BFFEE9AFEED92
:1011060099FDD0E0FBEF4E4D4C701222DB0302132B
:10111600A5EC2CFCEF33FFEE33FEED33FDED30E7AF
:10112600EB021380EF2BFFEE3AFEED39FDD0E0FB2C
:1011360050130BBB00030213A8ED13FDEE13FEEFD5
:0811460013FFEC13FC021380FF
:10114E00EC4D6011E8497017ED33EC3304600DE49B
:10115E00FCFFFEFD22E933E8330470F802139E1201
:10116E00136958046009E4CC248150062850090202
:10117E0013A82840030213A5C0E0EB4A7044B980BF
:10118E0006D0E0FB021394EF4E701CBD8008EBFFFF
:10119E00EAFEE9FD80EBE98DF0A4FEE5F0021237E0
:1011AE00E9CDF9EAFEEBFFEF89F0A4FCE5F0CE897C
:1011BE00F0A42EFFE435F0CD89F0A42DFEE435F039
:1011CE008067EF4E7005BD80D780C3EF8BF0A4AC67
:1011DE00F0EE8BF0A42CFCE435F0F8EF8AF0A42CA2
:1011EE00E5F038FCE433CB8DF0A42CFCE5F03BF8B5
:1011FE00EE8AF0A42CFCE5F038F8E433CF89F0A4A5
:10120E002CFCE5F038CF3400CE89F0A42FFFE5F0AA
:10121E003EFEE433C98DF0A42EFEE5F039CD8AF002
:10122E00A42FFFE5F03EFEE43DFD33D0E0FB50077A
:10123E000BBB000F0213A8EC2CFCEF33FFEE33FEBA
:06124E00ED33FD021380E8
:101254000213A8EC5D046005E85904700302139EB0
:10126400121369580460F6EC4860F2EC7004FDFE59
:10127400FF22C860DB2481C85009C398600250066D
:101284000213A59850CAF582E9294B4A7005AB822E
:1012940002139475F0007C1A7880C3EF9BEE9AEDEC
:1012A40099400DC3EF9BFFEE9AFEED99FDE842F0E5
:1012B400DC23ACF0D0E0FFD0E0FED0E0FDAB822038
:1012C400E7101BEB60BAEC2CFCEF33FFEE33FEEDC2
:1012D40033FD021380E803F830E705C0F075F00031
:1012E400EF2FFFEE33FEED33FD40B830E7C280AAA6
:1012F40075F020800E75F010800575F0087D007E75
:10130400007F003392D530D50312158EEC33401094
:10131400EF33FFEE33FEED33FDEC33FCD5F0ED227D
:0E132400E5F0247EA2D513CC92E7CDCEFF22B9
:10133200EDD2E7CD33EC3392D524814006E4FFFEB3
:10134200FDFC22FCE4CFCECDCC24E0501174FF8012
:10135200EDC3CC13CCCD13CDCE13CECF13CF0470AF
:07136200F030D5DE02158E0C
:10136900E9D2E7C933E833F892D5EDD2E7CD33ECCA
:0713790033FC5002B2D52243
:10138000EC30E7100FBF000C0EBE00080DBD0004CE
:101390000BEB6014A2D5EB13FCED92E7FD2274FF7A
:1013A000FCFDFEFF22E480F8A2D574FF13FC7D80D3
:0313B000E480EFE7
:1013B300BB010689828A83E0225002E722BBFE0238
:0913C300E32289828A83E493226B
:1013CC00EF8DF0A4A8F0CF8CF0A428CE8DF0A42E35
:0213DC00FE22EF
:1013DE00BC000BBE0029EF8DF084FFADF022E4CCF3
:1013EE00F875F008EF2FFFEE33FEEC33FCEE9DECBC
:1013FE00984005FCEE9DFE0FD5F0E9E4CEFD22ED02
:10140E00F8F5F0EE8420D21CFEADF075F008EF2F4B
:10141E00FFED33FD4007985006D5F0F222C398FD3C
:05142E000FD5F0EA22D9
:10143300C5F0F8A3E028F0C5F0F8E5821582700244
:061443001583E038F022E1
:0D144900EF2BFFEE3AFEED39FDEC38FC22F2
:0E145600C3EF9BFFEE9AFEED99FDEC98FC2291
:10146400E88FF0A4CC8BF0A42CFCE98EF0A42CFC27
:101474008AF0EDA42CFCEA8EF0A4CDA8F08BF0A4A5
:101484002DCC3825F0FDE98FF0A42CCD35F0FCEB04
:101494008EF0A4FEA9F0EB8FF0A4CFC5F02ECD39C9
:0F14A400FEE43CFCEAA42DCE35F0FDE43CFC2236
:1014B30075F008758200EF2FFFEE33FECD33CDCCF0
:1014C30033CCC58233C5829BED9AEC99E582984073
:1014D3000CF582EE9BFEED9AFDEC99FC0FD5F0D650
:1014E300E4CEFBE4CDFAE4CCF9A88222B800C1B97A
:1014F3000059BA002DEC8BF084CFCECDFCE5F0CBB8
:10150300F97818EF2FFFEE33FEED33FDEC33FCEBF0
:1015130033FB10D703994004EB99FB0FD8E5E4F9AB
:10152300FA227818EF2FFFEE33FEED33FDEC33FC98
:10153300C933C910D7059BE99A4007EC9BFCE99A8C
:10154300F90FD8E0E4C9FAE4CCFB2275F010EF2FD1
:10155300FFEE33FEED33FDCC33CCC833C810D707D1
:101563009BEC9AE899400AED9BFDEC9AFCE899F80C
:0E1573000FD5F0DAE4CDFBE4CCFAE4C8F9229F
:105E8F00C2D5E830E70FB2D5E4C39BFBE49AFAE43E
:105E9F0099F9E498F8EC30E717B2D5125EC51214F1
:105EAF00EFE4C39BFBE49AFAE499F9E498F88003D2
:105EBF001214EF30D50DE4C39FFFE49EFEE49DFD69
:045ECF00E49CFC2231
:0D158100EF4BFFEE4AFEED49FDEC48FC2269
:0E158E00C3E49FFFE49EFEE49DFDE49CFC226E
:10159C00EB9FF5F0EA9E42F0E99D42F0EC6480C8C6
:0615AC0064809845F02266
:1015B200EB9FF5F0EA9E42F0E99D42F0E89C45F08F
:0115C2002206
:1015C300E8600FECC313FCED13FDEE13FEEF13FF06
:0315D300D8F1222A
:1015D600E86010ECA2E713FCED13FDEE13FEEF132B
:0415E600FFD8F02218
:1015EA00E8600FEFC333FFEE33FEED33FDEC33FC5F
:0315FA00D8F12203
:0C15FD00E0FCA3E0FDA3E0FEA3E0FF2261
:0C160900E0F8A3E0F9A3E0FAA3E0FB2264
:0C161500ECF0A3EDF0A3EEF0A3EFF02248
:10162100A8828583F0D083D0821216381216381220
:101631001638121638E473E493A3C583C5F0C58345
:10164100C8C582C8F0A3C583C5F0C583C8C582C813
:011651002276
:0C165200A42582F582E5F03583F58322A3
:10165E00D083D082F8E4937012740193700DA3A31B
:10166E0093F8740193F5828883E47374029368602F
:06167E00EFA3A3A380DF2F
:10168400EC8EF0A4CCC5F0CCCDF8EFA4CEC5F02DF3
:10169400FDE43CFCE8A42EC8C5F03DFDE43CFCEFB1
:0D16A400A4FFE5F028FEE43DFDE43CFC223F
:08679E00EC30E70312158E2216
:00000001FF
